:1000000084EF26F000000000000000000000000067
:1000100000000000000000000000000000000000E0
:1000200000000000000000000000000000000000D0
:1000300000000000000000000000000000000113AC
:100040000000000000002D1500000000000000006E
:1000500000000000000000000000000000000000A0
:100060000000000000000000000000000000000090
:100070000000000000000000000000000000000080
:100080000000000000000000000000000000000070
:100090000000000000000000000000000000000060
:0C00A00000000000000000000000000054
:0C00AC00000E3D01F9BF010E006E1200B5
:0C00B800000E3D01E1BF010E006E1200C1
:0400C400F3DF120054
:0400C800F7DF12004C
:1000CC00FBDF005202E10000FBD76000DBF6EAFD2B
:0200DC00120010
:1000DE00F4DF005202E10000FBD76000DBF6D2FD38
:0200EE001200FE
:0E00F000026A016A006A086A036A000E1200C2
:1000FE000B820BAE89EF00F003680268016800689E
:08010E000A360232FF0E120056
:080116000AAE029E000E120069
:10011E000B840BAE9AEF00F0010E036E026A016AB9
:0A012E00006A0A360232FF0E1200CA
:08013800B5C1B6F1D0DF1200E1
:100140000CB0E2EF00F00CA288EF01F00E6A000E96
:100150000264F9EF00F0F00E0214D8A4C4EF00F02E
:10016000023A01380F0B02260138F00B016E0038FD
:100170000F0B01260038F00B006E08380F0B00261D
:100180000838F00B086E0E84D89002BEDDEF00F048
:1001900008360036013602360E2A02BEDDEF00F0C8
:1001A00008360036013602360E2A02BEDDEF00F0B8
:1001B00008360036013602360E2A0E5003647EEFF2
:1001C00001F0035E0BBC08AE83EF01F0D880800E17
:1001D00008640030000E002201220222D8A083EF22
:1001E00001F0023201320032034A88EF01F083EF5E
:1001F00001F001C002F000C001F008C000F0086A80
:10020000000E0E86026430EF01F0F00E0214D8A446
:1002100018EF01F0023A01380F0B02260138F00BFB
:10022000016E00380F0B01260038F00B006E0E84B3
:10023000D89002BEDDEF00F00036013602360E2AFD
:1002400002BEDDEF00F00036013602360E2A02BE95
:10025000DDEF00F00036013602360E2ADDEF00F049
:1002600001C002F000C001F0006A000E0E960E8878
:1002700002645DEF01F0F00E0214D8A448EF01F023
:10028000023A01380F0B02260138F00B016E0E8482
:10029000D89002BEDDEF00F0013602360E2A02BE13
:1002A000DDEF00F0013602360E2A02BEDDEF00F06F
:1002B000013602360E2ADDEF00F001C002F0016ABD
:1002C000000E0E8602648DEF01F0F00E0214D8A429
:1002D0006CEF01F0023A0E84D89002BEDDEF00F020
:1002E00002360E2A02BEDDEF00F002360E2A02BEF2
:1002F000DDEF00F002360E2ADDEF00F0010E0C6E8D
:100300000EDF90EF01F0020E0C6E05DF90EF01F0B2
:10031000040E0C6EF4DE90EF01F0080E0C6EE8DEB9
:020320001200C9
:08032200B5C1B6F1D2DE1200F4
:0E032A00550E3A01BF6FAA0EBF6FBF811200C1
:08033800B5C1B6F1C7DE1200E9
:0E034000550E3A01BF6FAA0EBF6FBF9112009B
:08034E00B5C1B6F1C5DE1200D5
:080356000B6A0B86FF0E12007A
:10035E00086A096A000E0762036437EF02F0025062
:10036E0006180A6E075003267E0ED8A0C5EF01F0C0
:10037E00035ED8B03BEF02F0C9EF01F0035ED8A0E8
:10038E003FEF02F0028E068E02C00EF001C00BF09F
:10039E0000C00DF0005004026F00D0FF0CF00150B1
:1003AE0005026F00D0FF00F06F00CCFF08F00402D2
:1003BE00F3500C26F4500822000E00220D500502B8
:1003CE00F3500C26F4500822000E002202500402B4
:1003DE00F3500826F450002202500502016A000E66
:1003EE000122F3500026F45001220D500602F35064
:1003FE000826F4500022026A000E012202220B503F
:10040E000602F3500026F4500122000E02220E5076
:10041E000602F3500126F450022202BE1FEF02F034
:10042E0008360036013602360306D8B43FEF02F026
:10043E0032EF02F0D880800E08640030000E0022E9
:10044E0001220222D8A032EF02F002320132003233
:10045E00034A3BEF02F00AAE029E000E41EF02F09D
:10046E00010E3FDE41EF02F0020E42DE41EF02F0DE
:06047E00040E4EDE120028
:100484000D6A086A0050D8B4000C04180A6E0ABE3B
:100494000D1E0B6A04AE02D0041E042A00AE02D064
:1004A400001E002A005004100A6E0ABE1FD0045019
:1004B400085E003600340836045008260036060E5E
:1004C4000C6E00340836045000B0085E00A0082604
:1004D40000360C2EF6D700A008260BB015D00DAEB2
:1004E400000C001E002A081E082A000C04AE09D0C5
:1004F40000BE04D00050086E006AF1D7006A002ADA
:10050400000C001E0B2AD3D7082A0450085CD8A478
:0E051400E6D7086A002A00AEE2D7FF0C1200FC
:100522000B800BAE9DEF02F0026A0AAEFF0E026E66
:0C053200016E006E0A360232FF0E12004D
:10053E00086A080E0C6E003408360450085ED8B0F7
:0E054E0002D00826D89000360C2EF5D71200E9
:10055C000101B151170802E2006A0ED3B251000A30
:10056C00D8A4B1D0B45301E0E5DE60D06000CFF682
:10057C0000FAA5D06000CFF601FAA1D06000CFF64A
:10058C0002FA9DD06000CFF603FA99D06000CFF646
:10059C0004FA95D06000CFF605FA91D06000CFF642
:1005AC0006FA8DD06000CFF607FA89D06000CFF63E
:1005BC0008FA85D06000CFF609FA81D06000CFF63A
:1005CC000AFA7DD06000CFF60BFA79D06000CFF636
:1005DC000CFA75D06000CFF60DFA71D06000CFF632
:1005EC000EFA6DD06000CFF60FFA69D06000CFF62E
:1005FC0010FA65D06000CFF611FA61D06000CFF62A
:10060C0012FA5DD06000CFF613FA59D06000CFF625
:10061C0014FA55D06000CFF615FA51D06000CFF621
:10062C0016FA4DD06000CFF617FA49D00101B1513E
:10063C00000A9CE0B151010A9DE0B151020A9EE012
:10064C00B151030A9FE0B151040AA0E0B151050A6F
:10065C00A1E0B151060AA2E0B151070AA3E0B151E1
:10066C00080AA4E0B151090AA5E0B1510A0AA6E0B2
:10067C00B1510B0AA7E0B1510C0AA8E0B1510D0A17
:10068C00A9E0B1510E0AAAE0B1510F0AABE0B15189
:10069C00100AACE0B151110AADE0B151120AAEE052
:1006AC00B151130AAFE0B151140AB0E0B151150ABF
:1006BC00B1E0B151160AB2E0B151170AB3E0010131
:1006CC00B45301E02CDE0101B251010AD8A451D17E
:1006DC00B45301E02FDEA4D06000C7F6C0FA45D1B8
:1006EC006000C7F6C1FA41D16000C7F6C2FA3DD12D
:1006FC006000C7F6C3FA39D16000C7F6C4FA35D129
:10070C006000C7F6C5FA31D16000C7F6C6FA2DD124
:10071C006000C7F6C7FA29D16000C7F6C8FA25D120
:10072C006000C7F6C9FA21D16000C7F6CAFA1DD11C
:10073C006000C7F6CBFA19D16000C7F6CCFA15D118
:10074C006000C7F6CDFA11D16000C7F6CEFA0DD114
:10075C006000C7F6CFFA09D16000C7F6D0FA05D110
:10076C006000C7F6D1FA01D16000C7F6D2FAFDD00D
:10077C006000C7F6D3FAF9D06000C7F6D4FAF5D00A
:10078C006000C7F6D5FAF1D06000C7F6D6FAEDD006
:10079C006000C7F6D7FAE9D06000C7F6D8FAE5D002
:1007AC006000C7F6D9FAE1D06000C7F6DAFADDD0FE
:1007BC006000C7F6DBFAD9D06000C7F6DCFAD5D0FA
:1007CC006000C7F6DDFAD1D06000C7F6DEFACDD0F6
:1007DC006000C7F6DFFAC9D06000C7F6E0FAC5D0F2
:1007EC006000C7F6E1FAC1D06000C7F6E2FABDD0EE
:1007FC006000C7F6E3FAB9D06000C7F6E4FAB5D0EA
:10080C006000C7F6E5FAB1D06000C7F6E6FAADD0E5
:10081C006000C7F6E8FAA9D06000C7F6E9FAA5D0DF
:10082C000101B351000AD8B457D7B351010AD8B457
:10083C0057D7B351020AD8B457D7B351030AD8B417
:10084C0057D7B351040AD8B457D7B351050AD8B403
:10085C0057D7B351060AD8B457D7B351070AD8B4EF
:10086C0057D7B351080AD8B457D7B351090AD8B4DB
:10087C0057D7B3510A0AD8B457D7B3510B0AD8B4C7
:10088C0057D7B3510C0AD8B457D7B3510D0AD8B4B3
:10089C0057D7B3510E0AD8B457D7B3510F0AD8B49F
:1008AC0057D7B351100AD8B457D7B351110AD8B48B
:1008BC0057D7B351120AD8B457D7B351130AD8B477
:1008CC0057D7B351140AD8B457D7B351150AD8B463
:1008DC0057D7B351160AD8B457D7B351170AD8B44F
:1008EC0057D7B351180AD8B457D7B351190AD8B43B
:1008FC0057D7B3511A0AD8B457D7B3511B0AD8B427
:10090C0057D7B3511C0AD8B457D7B3511D0AD8B412
:10091C0057D7B3511E0AD8B457D7B3511F0AD8B4FE
:10092C0057D7B351200AD8B457D7B351210AD8B4EA
:10093C0057D7B351220AD8B457D7B351230AD8B4D6
:10094C0057D7B351240AD8B457D7B351250AD8B4C2
:10095C0057D7B351260AD8B457D7B351270AD8B4AE
:10096C0057D7B351280AD8B457D70101B45301E073
:10097C00D6DCA8D00101B2B102D0C29001D0C280A5
:10098C00F9D00101B2B102D0C29201D0C282F2D030
:10099C000101B2B102D0C29401D0C284EBD00101EA
:1009AC00B2B102D0C29601D0C286E4D00101B2B17C
:1009BC0002D0C29801D0C288DDD00101B2B102D000
:1009CC00C29A01D0C28AD6D00101B2B102D0C29C67
:1009DC0001D0C28CCFD00101B2B102D0C29E01D0E5
:1009EC00C28EC8D00101B2B102D0C39001D0C38075
:1009FC00C1D00101B2B102D0C39201D0C382BAD02E
:100A0C000101B2B102D0C39401D0C384B3D00101AF
:100A1C00B2B102D0C39601D0C386ACD00101B2B141
:100A2C0002D0C39801D0C388A5D00101B2B102D0C5
:100A3C00C39A01D0C38A9ED00101B2B102D0C39C2B
:100A4C0001D0C38C97D00101B2B102D0C39E01D0AA
:100A5C00C38E90D00101B2B102D0C49001D0C48039
:100A6C0089D00101B2B102D0C49201D0C48282D02B
:100A7C000101B2B102D0C49401D0C4847BD0010175
:100A8C00B2B102D0C49601D0C48674D00101B2B107
:100A9C0002D0C49801D0C4886DD00101B2B102D08B
:100AAC00C49A01D0C48A66D00101B2B102D0C49CF0
:100ABC0001D0C48C5FD00101B2B102D0C49E01D070
:100ACC00C48E58D00101B151000AD8B453D7B151DA
:100ADC00010AD8B456D7B151020AD8B459D7B1517A
:100AEC00030AD8B45CD7B151040AD8B45FD7B1515A
:100AFC00050AD8B462D7B151060AD8B465D7B1513A
:100B0C00070AD8B468D7B151080AD8B46BD7B15119
:100B1C00090AD8B46ED7B1510A0AD8B471D7B151F9
:100B2C000B0AD8B474D7B1510C0AD8B477D7B151D9
:100B3C000D0AD8B47AD7B1510E0AD8B47DD7B151B9
:100B4C000F0A81E0B151100A85E0B151110A89E018
:100B5C00B151120A8DE0B151130A91E0B151140A4E
:100B6C0095E0B151150A99E0B151160A9DE0B151C9
:0A0B7C00170AA1E0FF0E006E120040
:100B8600025006180E6E086A096A0B6A035007645B
:100B9600B6EF06F006500A6E068E028E03500B6EF6
:100BA6000750036E000E0B6406EF06F00B50075E4F
:100BB600D8B4A7EF06F0070E076475EF06F0075ED8
:100BC60000C008F001C000F002C001F0026A074E42
:100BD600A7EF06F007644AEF06F0075E00C008F0CC
:100BE60001C000F0016A074EA7EF06F0076428EF80
:100BF60006F0075E00C008F0006A074EA7EF06F091
:100C060007640FEF06F00AC002F005C001F004C049
:100C160000F0086AD3EF07F0030E07641AEF06F038
:100C2600075E08380F0B086E074EA7EF06F0D89040
:100C36000832074EA7EF06F0D8900832074EA7EF06
:100C460006F0D8900832A7EF06F0030E076439EFD6
:100C560006F0075E08380F0B086E0038F00B082602
:100C660000380F0B006E074EA7EF06F0D890003243
:100C76000832074EA7EF06F0D89000320832074E2A
:100C8600A7EF06F0D89000320832A7EF06F0030E61
:100C9600076461EF06F0075E08380F0B086E003830
:100CA600F00B082600380F0B006E0138F00B0026FB
:100CB60001380F0B016E074EA7EF06F0D8900132F0
:100CC60000320832074EA7EF06F0D8900132003204
:100CD6000832074EA7EF06F0D890013200320832EC
:100CE600A7EF06F0030E076492EF06F0075E0838DA
:100CF6000F0B086E0038F00B082600380F0B006E3D
:100D06000138F00B002601380F0B016E0238F00B8C
:100D1600012602380F0B026E074EA7EF06F0D89099
:100D26000232013200320832074EA7EF06F0D890A1
:100D36000232013200320832074EA7EF06F0D89091
:100D46000232013200320832096A000E0EAE9BEF03
:100D560007F0081E001E011E021E082A002201229C
:100D660002229BEF07F00750D8A4BCEF06F0D3EFA2
:100D760007F0096A02C00AF0028E068E0750035C6D
:100D8600076ED8B48EEF07F0070E07645CEF07F026
:100D9600075E0450096E0550046E0650056E066A1D
:100DA600074E8EEF07F0070E076431EF07F0075E78
:100DB6000450096E0550046E056A074E8EEF07F063
:100DC600070E07640FEF07F0075E0450096E046A0A
:100DD600074E8EEF07F0070E0764F6EF06F00AC01F
:100DE60002F0D3EF07F0030E076401EF07F0075E8A
:100DF60009380F0B096E074E8EEF07F0D8900932AF
:100E0600074E8EEF07F0D8900932074E8EEF07F0A7
:100E1600D89009328EEF07F0030E076420EF07F033
:100E2600075E09380F0B096E0438F00B09260438E3
:100E36000F0B046E074E8EEF07F0D890043209327E
:100E4600074E8EEF07F0D89004320932074E8EEF28
:100E560007F0D890043209328EEF07F0030E0764CC
:100E660048EF07F0075E09380F0B096E0438F00BE0
:100E7600092604380F0B046E0538F00B04260538D6
:100E86000F0B056E074E8EEF07F0D8900532043231
:100E96000932074E8EEF07F0D89005320432093238
:100EA600074E8EEF07F0D8900532043209328EEFE6
:100EB60007F0030E076479EF07F0075E09380F0B9A
:100EC600096E0438F00B092604380F0B046E05383A
:100ED600F00B042605380F0B056E0638F00B0526B9
:100EE60006380F0B066E074E8EEF07F0D8900632C7
:100EF600053204320932074E8EEF07F0D8900632DB
:100F0600053204320932074E8EEF07F0D8900632CA
:100F1600053204320932086A000E0EAE9BEF07F066
:100F2600091E041E051E061E092A04220522062283
:100F360009500826045000220550012206500222BC
:100F46000EBEB2EF07F0D8A0C1EF07F002320132B1
:100F560000320832033EC1EF07F0CDEF07F0D8B0FC
:100F6600C7EF07F0000E081E001E011E021E082A0B
:100F76000022012202220A7EC7EF07F0010E0C6E44
:100F8600A0EC00F0D5EF07F0020E0C6EA0EC00F01E
:100F9600D5EF07F0040E0C6E7FEC00F0D5EF07F0EE
:060FA600000E0C6E1200AB
:100FAC00D250026ED29E0500FF6A0150FE6E0050B8
:080FBC00FD6E02BED28E120090
:100FC4000134083609360450085E0550D8A0053CA3
:100FD400095E003601360F0E0C6E013408360936F0
:100FE400045000A006D0085E0550D8A0053C095E58
:100FF40005D008260550D8B0053C09260036013630
:101004000C2EEBD700B006D0045008260550D8B0FB
:08101400053C09260000120052
:10101C00600083F5E1FF600087F5E2FF6000B3F646
:0E102C00E6FF5EC100F05FC101F0BADF120006
:10103A00ACC1B1F1ADC1B2F1AEC1B3F1010E010162
:08104A00B46FAEEC02F01200DD
:0A105200750E0D6E0D2EFED7120074
:10105C000B6A0C6A0A6A086A0350D8B4B6EF08F037
:10106C00028E9E0E035E03BE41EF08F0D8B441EF32
:10107C0008F0A6EF08F0036C080E035CD8A073EF21
:10108C0008F0036E083600C008F001C000F002C082
:10109C0001F0026A080E035CD8A073EF08F0036E2F
:1010AC00083600C008F001C000F0016A080E035CAD
:1010BC00D8A073EF08F0036E083600C008F0006A81
:1010CC00080E035CD8A073EF08F0036E0836086AAC
:1010DC000350D8A4D8907FEF08F00350D8B47FEF1A
:1010EC0008F0D8900232013200320832032E77EF2A
:1010FC0008F00BBC08A090EF08F0D8A090EF08F017
:10110C00082AD8B4002AD8B4012AD8B4022A02BEBC
:10111C00BAEF08F00AAEB6EF08F0021E011E001E70
:10112C00081E082AD8B4002AD8B4012AD8B4022A36
:10113C00B6EF08F0026A016A006A086AB6EF08F0B6
:10114C000B800BAEC0EF08F0026A0AAEC0EF08F0DD
:10115C00026E016E006E086E0A360232C0EF08F0A5
:10116C00000E0C6AC1EF08F0010E0C6E91EC02F04F
:10117C00C1EF08F0FF0E0250036E0150026E0050DA
:08118C00016E0850006E120014
:101194000A6A0350D8A40A800750D8A40A820A50C5
:1011A400D8B42DEF09F0030AD8B4E6EF08F00AB07A
:1011B400E1EF08F006AE2BEF09F029EF09F002AEDB
:1011C40029EF09F02BEF09F00250800B0A6E029E02
:1011D4000650800B069E0A18D8B4F7EF08F00A50A0
:1011E400D8B429EF09F02BEF09F00750035CD8B409
:1011F40001EF09F0D8A01DEF09F023EF09F0065024
:10120400025CD8B40BEF09F0D8A01DEF09F023EF6E
:1012140009F00550015CD8B415EF09F0D8A01DEF12
:1012240009F023EF09F00450005CD8B42DEF09F065
:10123400D8B023EF09F00A52D8B42BEF09F029EF04
:1012440009F00A52D8B429EF09F02BEF09F0D8803D
:0E1254001200D8901200D880D8841200120028
:101262000050086E0150006E0250016E0350026E73
:10127200036A0B6A0C6A9E0E036E0A6A020E0C6EF9
:06128200A0EC00F01200D8
:1012880003500718D8A458EF09F002500618D8A43C
:1012980058EF09F001500518D8A458EF09F000508C
:0E12A8000418D8B4D8841200D8941200120092
:1012B600800E0101AC19006E800E000A005CD8B0E9
:1012C60085D1AC510008016E01C0ACF1800E011849
:1012D600006E800E6E0A005CD8A0CCD0640E046E40
:1012E600ACC100F042EC02F0120E0024056E000EB6
:1012F60000BEFF0E066E000E062205C000F006C0F8
:1013060001F0000E06BEFF0E026E036E0036009060
:1013160001360236033600360090013602360336B1
:10132600A80E0024F66E550E0120F76E000E022060
:10133600F86E09006F00D4FFADF109006F00D4FF0D
:10134600AEF109006F00D4FFAFF109006F00D4FFC2
:10135600B0F1640E046EACC100F042EC02F008C0BD
:1013660000F00A0E046E42EC02F0090E0024056E2F
:10137600000E00BEFF0E066E000E062205C000F02F
:1013860006C001F0000E06BEFF0E026E036E0036AA
:1013960000900136023603360036009001360236DA
:1013A6000336A80E0024F66E550E0120F76E000EC9
:1013B6000220F86E09006F00D4FF00F009006F00EC
:1013C600D4FF01F009006F00D4FF02F009006F009E
:1013D600D4FF03F0ADC104F0AEC105F0AFC106F015
:1013E600B0C107F0AFEC01F000C0ADF101C0AEF145
:1013F60002C0AFF103C0B0F10A0E046EACC100F03A
:1014060042EC02F008C000F000C001F0000E00BE81
:10141600FF0E026E036E046E01360190023603362D
:10142600043601360190023603360436A80E01242E
:10143600F66E550E0220F76E000E0320F86E0900B8
:101446006F00D4FF00F009006F00D4FF01F009001F
:101456006F00D4FF02F009006F00D4FF03F0ADC1A6
:1014660004F0AEC105F0AFC106F0B0C107F0AFECB5
:1014760001F02BD2800E0A0A006E800EAC19005CB9
:1014860079E20A0E046EACC100F042EC02F0090EDD
:101496000024056E000E00BEFF0E066E000E06222C
:1014A60005C000F006C001F0000E06BEFF0E026E7B
:1014B600036E003600900136023603360036009081
:1014C600013602360336A80E0024F66E550E0120AC
:1014D600F76E000E0220F86E09006F00D4FFADF122
:1014E60009006F00D4FFAEF109006F00D4FFAFF121
:1014F60009006F00D4FFB0F10A0E046EACC100F013
:1015060042EC02F008C000F000C001F0000E00BE80
:10151600FF0E026E036E046E01360190023603362C
:10152600043601360190023603360436A80E01242D
:10153600F66E550E0220F76E000E0320F86E0900B7
:101546006F00D4FF00F009006F00D4FF01F009001E
:101556006F00D4FF02F009006F00D4FF03F0ADC1A5
:1015660004F0AEC105F0AFC106F0B0C107F0AFECB4
:1015760001F0ABD1ACC100F0000EACBFFF0E016EA6
:10158600026E036E003600900136023603360036D0
:101596000090013602360336A80E0024F66E550E6C
:1015A6000120F76E000E0220F86E09006F00D4FFCE
:1015B60000F009006F00D4FF01F009006F00D4FFAE
:1015C60002F009006F00D4FF03F07FD1800EAC1942
:1015D600006E800E6E0A005CD8A0CCD0640E046E3D
:1015E600ACC100F042EC02F0120E0024056E000EB3
:1015F60000BEFF0E066E000E062205C000F006C0F5
:1016060001F0000E06BEFF0E026E036E003600905D
:1016160001360236033600360090013602360336AE
:10162600DC0E0024F66E550E0120F76E000E022029
:10163600F86E09006F00D4FFADF109006F00D4FF0A
:10164600AEF109006F00D4FFAFF109006F00D4FFBF
:10165600B0F1640E046EACC100F042EC02F008C0BA
:1016660000F00A0E046E42EC02F0090E0024056E2C
:10167600000E00BEFF0E066E000E062205C000F02C
:1016860006C001F0000E06BEFF0E026E036E0036A7
:1016960000900136023603360036009001360236D7
:1016A6000336DC0E0024F66E550E0120F76E000E92
:1016B6000220F86E09006F00D4FF00F009006F00E9
:1016C600D4FF01F009006F00D4FF02F009006F009B
:1016D600D4FF03F0ADC104F0AEC105F0AFC106F012
:1016E600B0C107F0AFEC01F000C0ADF101C0AEF142
:1016F60002C0AFF103C0B0F10A0E046EACC100F037
:1017060042EC02F008C000F000C001F0000E00BE7E
:10171600FF0E026E036E046E01360190023603362A
:10172600043601360190023603360436DC0E0124F7
:10173600F66E550E0220F76E000E0320F86E0900B5
:101746006F00D4FF00F009006F00D4FF01F009001C
:101756006F00D4FF02F009006F00D4FF03F0ADC1A3
:1017660004F0AEC105F0AFC106F0B0C107F0AFECB2
:1017760001F0ABD0800E0A0A006E800EAC19005C38
:1017860079E20A0E046EACC100F042EC02F0090EDA
:101796000024056E000E00BEFF0E066E000E062229
:1017A60005C000F006C001F0000E06BEFF0E026E78
:1017B600036E00360090013602360336003600907E
:1017C600013602360336DC0E0024F66E550E012075
:1017D600F76E000E0220F86E09006F00D4FFADF11F
:1017E60009006F00D4FFAEF109006F00D4FFAFF11E
:1017F60009006F00D4FFB0F10A0E046EACC100F010
:1018060042EC02F008C000F000C001F0000E00BE7D
:10181600FF0E026E036E046E013601900236033629
:10182600043601360190023603360436DC0E0124F6
:10183600F66E550E0220F76E000E0320F86E0900B4
:101846006F00D4FF00F009006F00D4FF01F009001B
:101856006F00D4FF02F009006F00D4FF03F0ADC1A2
:1018660004F0AEC105F0AFC106F0B0C107F0AFECB1
:1018760001F02BD0ACC100F0000EACBFFF0E016E24
:10188600026E036E003600900136023603360036CD
:101896000090013602360336DC0E0024F66E550E35
:1018A6000120F76E000E0220F86E09006F00D4FFCB
:1018B60000F009006F00D4FF01F009006F00D4FFAB
:0C18C60002F009006F00D4FF03F01200D4
:0818D200067EC3EC05F01200D4
:1018DA000450000A08E10550000A05E1FF0E006EF7
:1018EA007F0E016E58D00D6A096A086A015000100D
:1018FA00D8B4000C015005180A6E0ABE0D1E0B6AF8
:10190A0005AE05D0041E051E042AD8B4052A01AE68
:10191A0005D0001E011E002AD8B4012A0150051064
:10192A000A6E0ABE10D0E2EC07F00BB020D00DAE62
:10193A00000C001E011E002AD8B4012A081E091E26
:10194A00082AD8B4092A000C05AE0DD001BE07D06A
:10195A000150096E0050086E016A006AE8D7016AF0
:10196A00006A002A000C011E001E0B2ADDD7082A75
:10197A00D8B4092A0450085CD8A4D9D70550095C00
:10198A00D8A4D5D7096A086A002AD8B4012A01AEB0
:08199A00CED70000FF0C120083
:1019A2006E0E0101AC5DD8A0D6D0640E046EACC13F
:1019B20000F09FEC02F0120E0024056E066A000E83
:1019C200062205C000F006C001F0000E06BEFF0EA2
:1019D200026E036E00360090013602360336003680
:1019E2000090013602360336A80E0024F66E550E1C
:1019F2000120F76E000E0220F86E09006F00D4FF7E
:101A020000F009006F00D4FF01F009006F00D4FF5D
:101A120002F009006F00D4FF03F0000E046E000E06
:101A2200056E000E066E7E0E076EAFEC01F000C072
:101A3200ADF101C0AEF102C0AFF103C0B0F1640E6E
:101A4200046EACC100F09FEC02F008C000F00A0E78
:101A5200046E9FEC02F0090E0024056E066A000E69
:101A6200062205C000F006C001F0000E06BEFF0E01
:101A7200026E036E003600900136023603360036DF
:101A82000090013602360336A80E0024F66E550E7B
:101A92000120F76E000E0220F86E09006F00D4FFDD
:101AA20000F009006F00D4FF01F009006F00D4FFBD
:101AB20002F009006F00D4FF03F0ADC104F0AEC123
:101AC20005F0AFC106F0B0C107F0AFEC01F000C005
:101AD200ADF101C0AEF102C0AFF103C0B0F10A0E28
:101AE200046EACC100F09FEC02F008C000F000C030
:101AF20001F0000E026E036E046E01360190023692
:101B02000336043601360190023603360436A80E37
:101B12000124F66E550E0220F76E000E0320F86EB9
:101B220009006F00D4FF00F009006F00D4FF01F03C
:101B320009006F00D4FF02F009006F00D4FF03F028
:101B4200ADC104F0AEC105F0AFC106F0B0C107F0FF
:101B5200AFEC01F0BDD0AC510A08D8B086D00A0E65
:101B6200046EACC100F09FEC02F0090E0024056E79
:101B7200066A000E062205C000F006C001F0000E43
:101B820006BEFF0E026E036E00360090013602366C
:101B9200033600360090013602360336A80E0024C2
:101BA200F66E550E0120F76E000E0220F86E090047
:101BB2006F00D4FF00F009006F00D4FF01F00900AC
:101BC2006F00D4FF02F009006F00D4FF03F0000E93
:101BD200046E000E056E000E066E7E0E076EAFECF2
:101BE20001F000C0ADF101C0AEF102C0AFF103C01F
:101BF200B0F10A0E046EACC100F09FEC02F008C016
:101C020000F000C001F0000E026E036E046E013699
:101C1200019002360336043601360190023603364D
:101C22000436A80E0124F66E550E0220F76E000E41
:101C32000320F86E09006F00D4FF00F009006F0066
:101C4200D4FF01F009006F00D4FF02F009006F0019
:101C5200D4FF03F0ADC104F0AEC105F0AFC106F090
:101C6200B0C107F0AFEC01F033D0ACC100F0000E10
:101C7200016E026E036E00360090013602360336A4
:101C820000360090013602360336A80E0024F66EA6
:101C9200550E0120F76E000E0220F86E09006F004B
:101CA200D4FF00F009006F00D4FF01F009006F00BB
:101CB200D4FF02F009006F00D4FF03F0000E046E9F
:101CC200000E056E000E066E7E0E076EAFEC01F082
:021CD2001200FE
:101CD4000101AC51390806E3300EAC5D03E3010E9B
:081CE400006E01D0006A12003D
:101CEC000450000A12E10550000A0FE10650000AE8
:101CFC000CE10750000A09E1FF0E006EFF0E016EA9
:101D0C007F0E026EFF0E036EA8D0086A096A075098
:101D1C00D8B421EF0FF00350D8B426EF0FF00250D7
:101D2C0006180A6E028E068E0E6A02C008F001C0FA
:101D3C000CF000C00DF004500D5E0550D8A0053C11
:101D4C000C5E0650D8A0063C085E086A0C6A0D6A48
:101D5C00D8A0B8EF0EF0D89002320132003208321F
:101D6C00010E0E6E0750035ED8A0C5EF0EF07E0E6E
:101D7C000E240326D8B02BEF0FF0CBEF0EF07E0E17
:101D8C000E240326D8A030EF0FF0180E0B6E0D3674
:101D9C000C3608360036013602360E360450005E1C
:101DAC000550D8A0053C015E0650D8A0063C025E4A
:101DBC0006340E120EA0E6EF0EF00D80F1EF0EF0D1
:101DCC00045000260550D8B0053C01260650D8B06A
:101DDC00062802260D900B2ECDEF0EF017EF0FF00C
:101DEC00D8900036013602360E360450005E05508F
:101DFC00D8A0053C015E0650D8A0063C025E063415
:101E0C000E10010B0D26D8B00C2AD8B4082AD8A471
:101E1C0017EF0FF008320C320D32032AD8B42BEF27
:101E2C000FF00AAE089E0850026E0C50016E0D5059
:101E3C00006E33EF0FF0010EABEC01F033EF0FF04F
:101E4C00020E78EC00F033EF0FF0040E7FEC00F094
:0C1E5C0033EF0FF0080E8FEC00F01200C6
:101E68000B6A0C6A086A0350D8B4B8EF0FF002C0C6
:101E78000AF0028E9E0E035E03AEA8EF0FF0036C0D
:101E8800080E035CD8A075EF0FF0036E083600C08B
:101E980008F001C000F002C001F0026A080E035CFD
:101EA800D8A075EF0FF0036E083600C008F001C027
:101EB80000F0016A080E035CD8A075EF0FF0036EFE
:101EC800083600C008F0006A080E035CD8A075EF59
:101ED8000FF0036E0836086A0350D8A4D89081EF33
:101EE8000FF00350D8B481EF0FF0D89002320132CE
:101EF80000320832032E79EF0FF00BBC08A092EFE6
:101F08000FF0D8A092EF0FF0082AD8B4002AD8B45E
:101F1800012AD8B4022A02BEBCEF0FF00AAEB8EF0D
:101F28000FF0021E011E001E081E082AD8B4002A3F
:101F3800D8B4012AD8B4022AB8EF0FF0026A016AAD
:101F4800006A086AB8EF0FF00B800BAEC3EF0FF012
:101F5800026A0AAEC3EF0FF0026E016E006E086EE1
:101F68000A360232C3EF0FF00C6A000EC4EF0FF00E
:101F7800010E0C6E000E91EC02F0C4EF0FF0FF0E94
:101F88000250036E0150026E0050016E0850006E40
:021F9800120035
:101F9A000B6A0A6A096A086A0E6A03340836045028
:101FAA00085E0550D8A0053C095E0650D8A0063C3C
:101FBA000A5E0750D8A0073C0B5EE86AD8A0010E5B
:101FCA000E5E0336070E0C6E0334083609360A36DF
:101FDA000B360E36045003A012D0085E0550D8A066
:101FEA00053C095E0650D8A0063C0A5E0750D8A0F8
:101FFA00073C0B5EE86AD8A0010E0E5E11D00826D7
:10200A000550D8B0053C09260650D8B0063C0A2629
:10201A000750D8B0073C0B26E86AD8B0010E0E2646
:10202A0003360C2ED1D70234083609360A360B3657
:10203A000E36045003A012D0085E0550D8A0053C05
:10204A00095E0650D8A0063C0A5E0750D8A0073C95
:10205A000B5EE86AD8A0010E0E5E11D00826055064
:10206A00D8B0053C09260650D8B0063C0A260750C7
:10207A00D8B0073C0B26E86AD8B0010E0E26023605
:10208A00070E0C6E0234083609360A360B360E363F
:10209A00045002A012D0085E0550D8A0053C095E83
:1020AA000650D8A0063C0A5E0750D8A0073C0B5E33
:1020BA00E86AD8A0010E0E5E11D008260550D8B0E5
:1020CA00053C09260650D8B0063C0A260750D8B067
:1020DA00073C0B26E86AD8B0010E0E2602360C2EF3
:1020EA00D1D70134083609360A360B360E36045073
:1020FA0002A012D0085E0550D8A0053C095E065021
:10210A00D8A0063C0A5E0750D8A0073C0B5EE86AD6
:10211A00D8A0010E0E5E11D008260550D8B0053C95
:10212A0009260650D8B0063C0A260750D8B0073C04
:10213A000B26E86AD8B0010E0E260136070E0C6E81
:10214A000134083609360A360B360E36045001A019
:10215A0012D0085E0550D8A0053C095E0650D8A0EA
:10216A00063C0A5E0750D8A0073C0B5EE86AD8A076
:10217A00010E0E5E11D008260550D8B0053C09267E
:10218A000650D8B0063C0A260750D8B0073C0B26A2
:10219A00E86AD8B0010E0E2601360C2ED1D70034CB
:1021AA00083609360A360B360E36045001A012D00C
:1021BA00085E0550D8A0053C095E0650D8A0063C2A
:1021CA000A5E0750D8A0073C0B5EE86AD8A0010E49
:1021DA000E5E11D008260550D8B0053C09260650D7
:1021EA00D8B0063C0A260750D8B0073C0B26E86A46
:1021FA00D8B0010E0E260036070E0C6E00340836D3
:10220A0009360A360B360E36045000A012D0085E84
:10221A000550D8A0053C095E0650D8A0063C0A5EC7
:10222A000750D8A0073C0B5EE86AD8A0010E0E5EE4
:10223A0011D008260550D8B0053C09260650D8B05A
:10224A00063C0A260750D8B0073C0B26E86AD8B0E5
:10225A00010E0E2600360C2ED1D700B00ED0045037
:10226A0008260550D8B0053C09260650D8B0063CC9
:0C227A000A260750D8B0073C0B261200C3
:102286000B6A0A6A096A005004026F00D0FF09F05F
:102296006F00CCFF08F0015005026F00D0FF0BF075
:1022A6006F00CCFF0AF000500502F3500926F450E7
:1022B6000A22E86A0B2201500402F3500926F45060
:1022C6000A22E86A0B2208C000F009C001F00AC021
:0822D60002F00BC003F012003E
:1022DE0084C15AF185C15BF186C15CF187C15DF1A4
:1022EE0088C15EF189C15FF18AC160F18BC161F174
:1022FE008CC150F18DC151F18EC152F18FC153F18C
:10230E0090C154F191C155F192C156F193C157F15B
:02231E001200AB
:102320003F0E010184153E01F16F29EC08F0F881A0
:102330000000F8A101D0FDD76F00BCFB00F06F00DA
:06234000C0FB01F01200D9
:0C2346006F00A0F701F001C000F01200D1
:10235200010184510308D8A0846B85510308D8A0D9
:10236200856BF00E3D01F217010184513D01F2131C
:10237200300EF21385C100F0003600900036009056
:1023820000360090003600900050F413F38F1200D4
:102392000101876B600013F6E9FF600017F6EAFFA0
:1023A2006F00B8FF86F18651000A10E086C1ACF1D9
:1023B2000EEC08F00101872B87518425E96E000E8F
:0E23C2008521EA6E6F00B8FF86F1EDD712009C
:1023D0000C6A0E6A0250D8A401EF12F001C002F09C
:1023E00000C001F0006A0E860250D8A401EF12F07E
:1023F00001C002F0016A0E960E880250D8B413EFA5
:1024000012F00E50035ED8A4D8A019EF12F0D890A5
:1024100002BE1FEF12F0003601360236032E08EF1F
:1024200012F019EF12F0010E0C6E78EC00F023EFB1
:1024300012F0020E0C6E8FEC00F023EF12F0040E7F
:082440000C6E8BEC00F01200A1
:10244800160E0101AC6FAD6B130EAE6F1DEC08F0EC
:10245800170E0101AC6F010EAD6F250EAE6F1DECAE
:0424680008F0120066
:10246C000101A46BA56B986B996B86C100F087C1B9
:10247C0001F088C102F0010E8627000E8723882305
:10248C00600003F0F6FF600007F0F7FF60000BF050
:10249C00F8FF09006F00D4FF00F000C095F1005266
:1024AC00D8B4B3EF23F09551250A0EE0600013F673
:1024BC00E1FF600017F6E2FF600057F6E6FF844B81
:1024CC00852BA44BA52BD1D7966B976B986B996BDF
:1024DC0023D09887010E8627000E872388236DD082
:1024EC009881010E8627000E8723882366D0988357
:1024FC00010E8627000E872388235FD09987010E53
:10250C008627000E8723882358D09885010E8627AE
:10251C00000E8723882351D060001BF6F6FF600065
:10252C001FF6F7FF600023F6F8FF09006F00D4FFD9
:10253C0001F001502D0ACDE060001BF6F6FF6000A3
:10254C001FF6F7FF600023F6F8FF09006F00D4FFB9
:10255C0001F00150200AC4E060001BF6F6FF600099
:10256C001FF6F7FF600023F6F8FF09006F00D4FF99
:10257C0001F001502B0ABBE060001BF6F6FF600077
:10258C001FF6F7FF600023F6F8FF09006F00D4FF79
:10259C0001F00150230AB2E060001BF6F6FF600068
:1025AC001FF6F7FF600023F6F8FF09006F00D4FF59
:1025BC0001F00150300AA9E001D08AD798A301D0CC
:1025CC00989198A701D0989560001BF6F6FF6000D3
:1025DC001FF6F7FF600023F6F8FF09006F00D4FF29
:1025EC0000F0000E016E00C0ACF16AEC0EF000526F
:1025FC003DE0966B976B96C100F097C101F00A0E07
:10260C00046E000E056E39DE60001BF6F6FF6000EE
:10261C001FF6F7FF600023F6F8FF09006F00D4FFE8
:10262C0002F002500024966F000E0120976F300EBE
:10263C00965F000E975B010E8627000E872388237A
:10264C0060001BF6F6FF60001FF6F7FF600023F634
:10265C00F8FF09006F00D4FF00F0000E016E00C0FF
:10266C00ACF16AEC0EF00052C6E145D060001BF6EE
:10267C00F6FF60001FF6F7FF600023F6F8FF090075
:10268C006F00D4FF01F001502A0A35E1600027F6F3
:10269C00E9FF60002BF6EAFF6F00B8FF00F06F0057
:1026AC00B8FF01F0600003F0E9FF600007F0EAFFFB
:1026BC006F00B8FF96F16F00B8FF97F1600027F636
:1026CC00E9FF60002BF6EAFF020EEE24006E000E0E
:1026DC00EE20016E600027F6E1FF60002BF6E2FFB2
:1026EC00600003F0E6FF600007F0E6FF010E8627AE
:1026FC00000E8723882360001BF6F6FF60001FF690
:10270C00F7FF600023F6F8FF09006F00D4FF01F01B
:10271C0001502E0AD8A489D0010E8627000E8723DB
:10272C00882360001BF6F6FF60001FF6F7FF6000C1
:10273C0023F6F8FF09006F00D4FF01F001502A0ABC
:10274C0036E1600027F6E9FF60002BF6EAFF6F0028
:10275C00B8FF00F06F00B8FF01F0600003F0E9FF74
:10276C00600007F0EAFF6F00B8FF93F16F00B8FF4D
:10277C0094F1600027F6E9FF60002BF6EAFF020EE9
:10278C00EE24006E000EEE20016E600027F6E1FFD5
:10279C0060002BF6E2FF600003F0E6FF600007F03C
:1027AC00E6FF010E8627000E872388233DD0936B0E
:1027BC00946B60001BF6F6FF60001FF6F7FF6000DD
:1027CC0023F6F8FF09006F00D4FF00F0000E016E35
:1027DC0000C0ACF16AEC0EF0005226E093C100F0A0
:1027EC0094C101F00A0E046E000E056E46DD600009
:1027FC001BF6F6FF60001FF6F7FF600023F6F8FFEC
:10280C0009006F00D4FF02F002500024936F000EF9
:10281C000120946F300E935F000E945B010E86279F
:10282C00000E87238823C5D703D0936B946B9989AB
:10283C0086C100F087C101F088C102F0010E862725
:10284C00000E87238823600003F0F6FF600007F07A
:10285C00F7FF60000BF0F8FF09006F00D4FF95F153
:10286C001DD1A4C100F0A5C101F0B7EF23F09889E8
:10287C00DFD7998552D1988B99814FD199834DD1BE
:10288C00988D4BD14AD1988B988F47D1600027F601
:10289C00E9FF60002BF6EAFF6F00B8FF00F06F0055
:1028AC00B8FF01F0600003F0E9FF600007F0EAFFF9
:1028BC006F00B8FFA0F16F00B8FFA1F1600027F620
:1028CC00E9FF60002BF6EAFF020EEE24006E000E0C
:1028DC00EE20016E600027F6E1FF60002BF6E2FFB0
:1028EC00600003F0E6FF600007F0E6FF000EA119A0
:1028FC0002E1000EA01904E13A0EA06F000EA16FC8
:10290C00A26BA36BA251A025E96EA351A121EA6E83
:10291C00EE520BE0010EA225006E000EA321016EFB
:10292C0000C0A2F101C0A3F1EDD7935194110AE0BC
:10293C00A351945D02E1A251935D04E293C1A2F113
:10294C0094C1A3F19751A35D02E19651A25D05E2FA
:10295C00A251965FA351975B02D0966B976B98B779
:10296C0018D096C100F097C101F0010E965F000ED1
:10297C00975B005001100DE0600013F6E1FF600062
:10298C0017F6E2FF200EE66E844B852BA44BA52B8D
:10299C00E8D7A2C102F0A3C103F0010EA25D006E44
:1029AC00000EA359016E00C0A2F101C0A3F10250A8
:1029BC0003101EE0600083F6E9FF600087F6EAFF73
:1029CC00600013F6E1FF600017F6E2FF6F00BBFF3B
:1029DC00E6FF844B852B010EA025006E000EA12175
:1029EC00016E00C0A0F101C0A1F1A44BA52BD1D761
:1029FC0098A718D096C100F097C101F0010E965F10
:102A0C00000E975B005001100DE0600013F6E1FF23
:102A1C00600017F6E2FF200EE66E844B852BA44B6C
:102A2C00A52BE8D722D5600027F6E9FF60002BF62E
:102A3C00EAFF6F00B8FF00F06F00B8FF01F0600014
:102A4C0003F0E9FF600007F0EAFF6F00B8FF95F1B3
:102A5C00600027F6E9FF60002BF6EAFF020EEE2479
:102A6C00006E000EEE20016E600027F6E1FF6000A4
:102A7C002BF6E2FF600003F0E6FF600007F0E6FFD4
:102A8C00950EA06F010EA16F010EA26F000EA36F29
:102A9C004CD7C00E9813000E99133FD09551000AD5
:102AAC00D8B4DFD695516C0AD8B4E1D695514C0AFE
:102ABC00D8B4DDD69551660AD8B4DBD69551450A03
:102ACC00D8B4D9D69551650AD8B4D6D69551670ADB
:102ADC00D8B4D4D695516F0AD8B4D2D69551640ACD
:102AEC00D8B4D0D69551690AD8B4CCD69551700AC1
:102AFC00D8B4C9D69551580AD8B4C5D69551780AC8
:102B0C00D8B4C2D69551730AD8B4C0D69551630ABD
:102B1C008AE09551750ABDE0B3D7000E9815006E8A
:102B2C009951070B016E00500110D8B4DEEF1EF066
:102B3C0099A904D0060E936F000E946F600027F6CF
:102B4C00E9FF60002BF6EAFF6F00B8FF00F06F00A2
:102B5C00B8FF01F0600003F0E9FF600007F0EAFF46
:102B6C006F00B8FF9AF16F00B8FF9BF16F00B8FFD0
:102B7C009CF16F00B8FF9DF1600027F6E9FF600043
:102B8C002BF6EAFF040EEE24006E000EEE20016E12
:102B9C00600027F6E1FF60002BF6E2FF600003F017
:102BAC00E6FF600007F0E6FF046A056A066A076A3A
:102BBC009AC100F09BC101F09CC102F09DC103F0D1
:102BCC00CAEC08F0010ED8B0000E006E005205E001
:102BDC009C7F030E9813000E99139E6B9F6B9AC1EA
:102BEC0000F09BC101F09CC102F09DC103F0046A8E
:102BFC00056A066A076A44EC09F0000ED8A4010EB7
:102C0C00006E0052D8B48AD09DC100F0016A026AED
:102C1C00036AFF0E0016000E01167E0E005E000EFB
:102C2C00015A00C09EF101C09FF1010E005E000E22
:102C3C00015A00C09EF101C09FF1030E046E000EFC
:102C4C00056E43EC11F000C09EF101C09FF10A0E1D
:102C5C00046E000E056E6DEC0CF000C09EF101C010
:102C6C009FF1800E0118026E800E025C02E1000ED4
:102C7C00005C05E2010E01019E5F000E9F5B0101ED
:102C8C009E510008AC6F5BEC09F09AC104F09BC13B
:102C9C0005F09CC106F09DC107F0AFEC01F000C03F
:102CAC00A0F101C0A1F102C0A2F103C0A3F1000E7A
:102CBC00046E000E056E000E066E7F0E076EA0C130
:102CCC0000F0A1C101F0A2C102F0A3C103F0CAEC53
:102CDC0008F0010ED8B0000E006E005205E0010E97
:102CEC009E5F000E9F5B1AD0000E046E000E056EE8
:102CFC00200E066E820E076EA0C100F0A1C101F07D
:102D0C00A2C102F0A3C103F0CAEC08F0000ED8B0C7
:102D1C00010E006E005202E09E4B9F2B800E006E47
:102D2C00800E9F19005C02E19E51000803E3010E26
:102D3C00956F02D09EC195F199B119D099A315D078
:102D4C00800E9F19006E7F0E005C02E1FC0E9E5DF2
:102D5C000BE3800E9F19006E800E9419005C02E14B
:102D6C0093519E5D01E201D002D0E4EF1AF0935131
:102D7C00941106E099A304D0010E935F000E945BAE
:102D8C009451000802E19351080803E2080E956F74
:102D9C0002D093C195F19AC100F09BC101F09CC186
:102DAC0002F09DC103F0046A056A066A076A44ECE6
:102DBC0009F0000ED8A4010E006E0052D8B453D105
:102DCC009EC1ACF15BEC09F000C004F001C005F051
:102DDC0002C006F003C007F09AC100F09BC101F0DD
:102DEC009CC102F09DC103F076EC0EF000C09AF18C
:102DFC0001C09BF102C09CF103C09DF101019551F2
:102E0C000008AC6F5BEC09F000C004F001C005F0E9
:102E1C0002C006F003C007F09AC100F09BC101F09C
:102E2C009CC102F09DC103F076EC0EF000C0A6F13F
:102E3C0001C0A7F102C0A8F103C0A9F1A6C19AF183
:102E4C00A7C19BF1A8C19CF1A9C19DF1A6C100F03D
:102E5C00A7C101F0A8C102F0A9C103F02EEC08F043
:102E6C0031EC09F000C004F001C005F002C006F01E
:102E7C0003C007F0A6C100F0A7C101F0A8C102F081
:102E8C00A9C103F069EC0CF0000E046E000E056E87
:102E9C00000E066E7E0E076ECAEC08F0000ED8B05F
:102EAC00010E006E00521AE09AC100F09BC101F0B5
:102EBC009CC102F09DC103F0000E046E000E056E65
:102ECC00000E066E7E0E076EC3EC05F000C09AF184
:102EDC0001C09BF102C09CF103C09DF19AC100F0AE
:102EEC009BC101F09CC102F09DC103F02EEC08F0D7
:102EFC0001019551010F096E0A6A000E0A2209C0E0
:102F0C0004F00AC005F0000E0ABEFF0E066E076E36
:102F1C00043604900536063607360436049005361A
:102F2C00063607366C0E0424F66E560E0520F76E28
:102F3C00000E0620F86E09006F00D4FF05F00900A2
:102F4C006F00D4FF06F009006F00D4FF07F00900F2
:102F5C006F00D4FF08F00850035C08E10750025CD6
:102F6C0005E10650015C02E10550005C1EE3010125
:102F7C009AC100F09BC101F09CC102F09DC103F00D
:102F8C00CD0E046ECC0E056E4C0E066E7B0E076ECF
:102F9C00AFEC01F000C09AF101C09BF102C09CF1B2
:102FAC0003C09DF19E4B9F2B5ED09AC100F09BC13C
:102FBC0001F09CC102F09DC103F02EEC08F095C10C
:102FCC0004F0000E056E066E076E0436049005368E
:102FDC0006360736043604900536063607366C0E70
:102FEC000424F66E560E0520F76E000E0620F86EC1
:102FFC0009006F00D4FF05F009006F00D4FF06F044
:10300C0009006F00D4FF07F009006F00D4FF08F02F
:10301C000850035C08E10750025C05E10650015CB6
:10302C0002E10550005C1FE201019AC100F09BC156
:10303C0001F09CC102F09DC103F0000E046E000E65
:10304C00056E200E066E820E076EAFEC01F000C00E
:10305C009AF101C09BF102C09CF103C09DF1010EDD
:10306C009E5F000E9F5B010199A393D099B791D0FD
:10307C00800E000A006E800E9419005C02E19351E0
:10308C000A0804E20A0E936F000E946F9AC100F0C6
:10309C009BC101F09CC102F09DC103F02EEC08F025
:1030AC0000C0A0F101C0A1F102C0A2F103C0A3F1C4
:1030BC00A051A111A211A31142E00A0E046E000E40
:1030CC00056E066E076EA0C100F0A1C101F0A2C191
:1030DC0002F0A3C103F0CDEC0FF008C000F009C062
:1030EC0001F00AC002F00BC003F0000E046E0318CE
:1030FC0008E10450021805E10450011802E10050E7
:10310C00000A1DE1010E935F000E945B0A0E046E23
:10311C00000E056E066E076EA0C100F0A1C101F095
:10312C00A2C102F0A3C103F0CDEC0FF000C0A0F1DE
:10313C0001C0A1F102C0A2F103C0A3F1B9D7800E66
:10314C009419006E800E005C02E19551935D21E2B2
:10315C009351955DAC6F5BEC09F000C004F001C0BD
:10316C0005F002C006F003C007F09AC100F09BC145
:10317C0001F09CC102F09DC103F076EC0EF000C092
:10318C009AF101C09BF102C09CF103C09DF193C167
:10319C0095F1050E01019325006E000E9421016E30
:1031AC000050965F0150975B9351941103E199B7CE
:1031BC0001D004D0010E965F000E975B030E98159C
:1031CC00006E99C101F0000E01160050011004E0D0
:1031DC00010E965F000E975B98A540D098A315D072
:1031EC0098A103D02D0E8B6F02D02B0E8B6F60002D
:1031FC0013F6E1FF600017F6E2FF60002FF6E6FF22
:10320C00844B852BA44BA52B0ED098A10CD0600021
:10321C0013F6E1FF600017F6E2FF200EE66E844B1A
:10322C00852BA44BA52B800E006E800E9719005C8D
:10323C0002E19651000811E2600013F6E1FF600014
:10324C0017F6E2FF300EE66E844B852BA44BA52BB4
:10325C00010E965F000E975BE6D741D098B71AD057
:10326C00800E006E800E9719005C02E196510008EA
:10327C0011E2600013F6E1FF600017F6E2FF200E8A
:10328C00E66E844B852BA44BA52B010E965F000E8E
:10329C00975BE6D798A315D098A103D02D0E8C6F11
:1032AC0002D02B0E8C6F600013F6E1FF600017F656
:1032BC00E2FF600033F6E6FF844B852BA44BA52B75
:1032CC000ED098A10CD0600013F6E1FF600017F649
:1032DC00E2FF200EE66E844B852BA44BA52B9AC1E6
:1032EC0000F09BC101F09CC102F09DC103F02EECDB
:1032FC0008F000C0A0F101C0A1F102C0A2F103C00E
:10330C00A3F195C100F0000E016E026E036E003643
:10331C000090013602360336003600900136023634
:10332C0003366C0E0024F66E560E0120F76E000E5E
:10333C000220F86E09006F00D4FF04F009006F0042
:10334C00D4FF05F009006F00D4FF06F009006F00F0
:10335C00D4FF07F0A0C100F0A1C101F0A2C102F09E
:10336C00A3C103F0CDEC0FF0300E0026600013F675
:10337C00E1FF600017F6E2FF600003F0E6FF844B0C
:10338C00852BA44BA52B9351941103E199B701D034
:10339C007AD0600013F6E1FF600017F6E2FF2E0E04
:1033AC00E66E844B852BA44BA52B9551935F000E99
:1033BC00945B955354E0950795C100F0000E016E97
:1033CC00026E036E0036009001360236033600366C
:1033DC0000900136023603366C0E0024F66E560E43
:1033EC000120F76E000E0220F86E09006F00D4FF6A
:1033FC0004F009006F00D4FF05F009006F00D4FF42
:10340C0006F009006F00D4FF07F0A0C100F0A1C1C5
:10341C0001F0A2C102F0A3C103F0CDEC0FF00A0E33
:10342C00046E000E056E066E076ECDEC0FF008C034
:10343C0000F009C001F00AC002F00BC003F0300E1E
:10344C000026600013F6E1FF600017F6E2FF600053
:10345C0003F0E6FF844B852BA44BA52BAAD79351E5
:10346C00941111E0600013F6E1FF600017F6E2FF23
:10347C00300EE66E844B852BA44BA52B010E935F6F
:10348C00000E945BECD798AB0DD0600013F6E1FF07
:10349C00600017F6E2FF450EE66E844B852BA44BBD
:1034AC00A52B0CD0600013F6E1FF600017F6E2FFCD
:1034BC00650EE66E844B852BA44BA52B800E9F19B5
:1034CC00006E800E005C02E1000E9E5D13E29E51C8
:1034DC0000089E6F9F51000E9F57600013F6E1FF8E
:1034EC00600017F6E2FF2D0EE66E844B852BA44B85
:1034FC00A52B0CD0600013F6E1FF600017F6E2FF7D
:10350C002B0EE66E844B852BA44BA52B0A0E046E5A
:10351C00000E056E9EC100F09FC101F06DEC0CF029
:10352C00300E0026600013F6E1FF600017F6E2FF94
:10353C00600003F0E6FF0101844B852BA44BA52B07
:10354C000A0E046E000E056E9EC100F09FC101F0C4
:10355C006DEC0CF008C000F009C001F0300E002634
:10356C00600013F6E1FF600017F6E2FF600003F065
:10357C00E6FF0101844B852BA44BA52B98A71CD0EF
:10358C00800E006E800E9719005C02E196510008C7
:10359C0013E2600013F6E1FF600017F6E2FF200E65
:1035AC00E66E844B852BA44BA52B010E965F000E6B
:1035BC00975B96519711EDE13BEF12F099A3F7D081
:1035CC00800E9F19006E800E005C02E1000E9E5D65
:1035DC000AE2010E9E5D006E000E9F59016E0050B6
:1035EC00935F0150945B9AC100F09BC101F09CC1A8
:1035FC0002F09DC103F02EEC08F000C0A0F101C058
:10360C00A1F102C0A2F103C0A3F1010E956F955177
:10361C000A0A38E095C100F0000E016E026E036ECE
:10362C000036009001360236033600360090013623
:10363C00023603366C0E0024F66E560E0120F76E21
:10364C00000E0220F86E09006F00D4FF01F0090093
:10365C006F00D4FF02F009006F00D4FF03F00900E3
:10366C006F00D4FF04F00450A35D08E10350A25D89
:10367C0005E10250A15D02E10150A05D01E202D022
:10368C00952BC5D79551935DAA6F000E9459AB6FCE
:10369C00AAC193F1ABC194F1A0C100F0A1C101F09A
:1036AC00A2C102F0A3C103F031EC09F000C004F098
:1036BC0001C005F002C006F003C007F09AC100F08B
:1036CC009BC101F09CC102F09DC103F069EC0CF0B0
:1036DC0000C0A6F101C0A7F102C0A8F103C0A9F176
:1036EC00AAC1ACF15BEC09F0A6C104F0A7C105F0CE
:1036FC00A8C106F0A9C107F0AFEC01F0000E046EF2
:10370C00000E056E000E066E7E0E076EC3EC05F005
:10371C002EEC08F000C0A0F101C0A1F102C0A2F192
:10372C0003C0A3F19351941142E00A0E046E000EF3
:10373C00056E066E076EA0C100F0A1C101F0A2C11A
:10374C0002F0A3C103F0CDEC0FF008C000F009C0EB
:10375C0001F00AC002F00BC003F0000E046E031857
:10376C0008E10450021805E10450011802E1005070
:10377C00000A1DE10A0E046E000E056E066E076E41
:10378C00A0C100F0A1C101F0A2C102F0A3C103F0DD
:10379C00CDEC0FF000C0A0F101C0A1F102C0A2F16C
:1037AC0003C0A3F1010E935F000E945BBBD7800E98
:1037BC00006E800E9419005C02E193510C0816E324
:1037CC0093C1ACF1D1EC0CF09AC104F09BC105F0A3
:1037DC009CC106F09DC107F0C3EC05F000C09AF146
:1037EC0001C09BF102C09CF103C09DF19AC100F095
:1037FC009BC101F09CC102F09DC103F0046A056AF3
:10380C00066A076A44EC09F0000ED8A4010E006E9B
:10381C000052D8B477D09AC100F09BC101F09CC182
:10382C0002F09DC103F02EEC08F0000E046E03189C
:10383C0008E10450021805E10450011802E100509F
:10384C00000A60E1800E006E800E9F19005C02E1A0
:10385C009E51010857E29EC1ACF15BEC09F000C02F
:10386C0004F001C005F002C006F003C007F09AC1D5
:10387C0000F09BC101F09CC102F09DC103F076ECFD
:10388C000EF05F0E046E700E056E090E066E810E44
:10389C00076ECAEC08F0010ED8B0000E006E005294
:1038AC0006E0090E01019E5F000E9F5B05D0010131
:1038BC00080E9E5F000E9F5B9EC1ACF15BEC09F0A5
:1038CC0000C004F001C005F002C006F003C007F010
:1038DC009AC100F09BC101F09CC102F09DC103F0A4
:1038EC0076EC0EF02EEC08F000C0A0F101C0A1F1B6
:1038FC0002C0A2F103C0A3F101019A6B9B6B9C6BFC
:10390C009D6B38D09AC100F09BC101F09CC102F0B4
:10391C009DC103F02EEC08F000C0A0F101C0A1F194
:10392C0002C0A2F103C0A3F1A0C100F0A1C101F03B
:10393C00A2C102F0A3C103F031EC09F000C004F005
:10394C0001C005F002C006F003C007F09AC100F0F8
:10395C009BC101F09CC102F09DC103F069EC0CF01D
:10396C0000C09AF101C09BF102C09CF103C09DF113
:10397C009E6B9F6B010E956F95510A0A38E095C1AD
:10398C0000F0000E016E026E036E003600900136E0
:10399C0002360336003600900136023603366C0EC2
:1039AC000024F66E560E0120F76E000E0220F86E03
:1039BC0009006F00D4FF01F009006F00D4FF02F082
:1039CC0009006F00D4FF03F009006F00D4FF04F06E
:1039DC000450A35D08E10350A25D05E10250A15D16
:1039EC0002E10150A05D01E202D0952BC5D79551A3
:1039FC009325006E000E9421016E9E5100269F515E
:103A0C0001220050965F0150975B99B704D09351F7
:103A1C00941101E104D0010E965F000E975B030E2A
:103A2C009815006E99C101F0000E0116005001109E
:103A3C0004E0010E965F000E975B98A540D098A30A
:103A4C0015D098A103D02D0E8D6F02D02B0E8D6F3B
:103A5C00600013F6E1FF600017F6E2FF600037F636
:103A6C00E6FF844B852BA44BA52B0ED098A10CD034
:103A7C00600013F6E1FF600017F6E2FF200EE66E21
:103A8C00844B852BA44BA52B800E006E800E9719B2
:103A9C00005C02E19651000811E2600013F6E1FFB0
:103AAC00600017F6E2FF300EE66E844B852BA44BBC
:103ABC00A52B010E965F000E975BE6D741D098B709
:103ACC001AD0800E006E800E9719005C02E19651A0
:103ADC00000811E2600013F6E1FF600017F6E2FF48
:103AEC00200EE66E844B852BA44BA52B010E965F06
:103AFC00000E975BE6D798A315D098A103D02D0E96
:103B0C008E6F02D02B0E8E6F600013F6E1FF6000FB
:103B1C0017F6E2FF60003BF6E6FF844B852BA44BC7
:103B2C00A52B0ED098A10CD0600013F6E1FF60001D
:103B3C0017F6E2FF200EE66E844B852BA44BA52BCB
:103B4C0095C100F09507005253E095C100F0000EAE
:103B5C00016E026E036E003600900136023603369B
:103B6C00003600900136023603366C0E0024F66ED9
:103B7C00560E0120F76E000E0220F86E09006F0041
:103B8C00D4FF04F009006F00D4FF05F009006F00AA
:103B9C00D4FF06F009006F00D4FF07F0A0C100F0BD
:103BAC00A1C101F0A2C102F0A3C103F0CDEC0FF052
:103BBC000A0E046E000E056E066E076ECDEC0FF04D
:103BCC0008C000F009C001F00AC002F00BC003F0FD
:103BDC00300E0026600013F6E1FF600017F6E2FFDE
:103BEC00600003F0E6FF844B852BA44BA52BA8D7D4
:103BFC00800E006E800E9F19005C02E19E51000841
:103C0C0011E2600013F6E1FF600017F6E2FF300EE0
:103C1C00E66E844B852BA44BA52B010E9E5F000EEC
:103C2C009F5BE6D7800E000A006E800E9419005C34
:103C3C0002E19351080803E2080E956F02D093C17C
:103C4C0095F19551935F000E945B955303E199B7F1
:103C5C0001D00CD0600013F6E1FF600017F6E2FF14
:103C6C002E0EE66E844B852BA44BA52B95C1ACF187
:103C7C005BEC09F09AC104F09BC105F09CC106F005
:103C8C009DC107F0AFEC01F034EC0FF000C0A0F1D7
:103C9C0001C0A1F102C0A2F103C0A3F1955354E0FD
:103CAC00950795C100F0000E016E026E036E003692
:103CBC00009001360236033600360090013602368B
:103CCC0003366C0E0024F66E560E0120F76E000EB5
:103CDC000220F86E09006F00D4FF04F009006F0099
:103CEC00D4FF05F009006F00D4FF06F009006F0047
:103CFC00D4FF07F0A0C100F0A1C101F0A2C102F0F5
:103D0C00A3C103F0CDEC0FF00A0E046E000E056E8D
:103D1C00066E076ECDEC0FF008C000F009C001F084
:103D2C000AC002F00BC003F0300E0026600013F640
:103D3C00E1FF600017F6E2FF600003F0E6FF844B42
:103D4C00852BA44BA52BAAD79351941111E060009D
:103D5C0013F6E1FF600017F6E2FF300EE66E844BBF
:103D6C00852BA44BA52B010E935F000E945BECD717
:103D7C0098A71CD0800E006E800E9719005C02E193
:103D8C009651000813E2600013F6E1FF600017F68D
:103D9C00E2FF200EE66E844B852BA44BA52B010E67
:103DAC00965F000E975B96519711EDE13BEF12F089
:103DBC00C00E9815016E99C102F0000E0216000E8D
:103DCC00021802E1000E0118D8A49ED098A937D091
:103DDC00600027F6E9FF60002BF6EAFF6F00B8FFE2
:103DEC0000F06F00B8FF01F0600003F0E9FF600025
:103DFC0007F0EAFF6F00B8FFA0F16F00B8FFA1F168
:103E0C006F00B8FFA2F16F00B8FFA3F1600027F6B6
:103E1C00E9FF60002BF6EAFF040EEE24006E000EA4
:103E2C00EE20016E600027F6E1FF60002BF6E2FF4A
:103E3C00600003F0E6FF600007F0E6FF3DD0600095
:103E4C0027F6E9FF60002BF6EAFF6F00B8FF00F0E1
:103E5C006F00B8FF01F0600003F0E9FF600007F0AD
:103E6C00EAFF6F00B8FF00F06F00B8FF01F0000E22
:103E7C0001BEFF0E026E036E00C0A0F101C0A1F1E5
:103E8C0002C0A2F103C0A3F1600027F6E9FF6000B5
:103E9C002BF6EAFF020EEE24006E000EEE20016EF1
:103EAC00600027F6E1FF60002BF6E2FF600003F0F4
:103EBC00E6FF600007F0E6FF800EA319006E800E8F
:103ECC00005C08E1000EA25D05E1000EA15D02E1BF
:103EDC00000EA05D18E2030E9813000E9913006AF1
:103EEC00016A026A036AA051005EA151015AA251F3
:103EFC00025AA351035A00C0A0F101C0A1F102C0A3
:103F0C00A2F103C0A3F16CD098A937D0600027F6BA
:103F1C00E9FF60002BF6EAFF6F00B8FF00F06F00BE
:103F2C00B8FF01F0600003F0E9FF600007F0EAFF62
:103F3C006F00B8FFA0F16F00B8FFA1F16F00B8FFE0
:103F4C00A2F16F00B8FFA3F1600027F6E9FF600053
:103F5C002BF6EAFF040EEE24006E000EEE20016E2E
:103F6C00600027F6E1FF60002BF6E2FF600003F033
:103F7C00E6FF600007F0E6FF33D0600027F6E9FFAC
:103F8C0060002BF6EAFF6F00B8FF00F06F00B8FF7F
:103F9C0001F0600003F0E9FF600007F0EAFF6F003A
:103FAC00B8FFA0F16F00B8FFA1F1000EA26FA36FD4
:103FBC00600027F6E9FF60002BF6EAFF020EEE2404
:103FCC00006E000EEE20016E600027F6E1FF60002F
:103FDC002BF6E2FF600003F0E6FF600007F0E6FF5F
:103FEC00000E941902E1000E93190FE1000E006E01
:103FFC00A31908E10050A21905E10050A11902E132
:10400C00A051000A02E1934B942BC00E9815006E40
:10401C0000C005F0BAD0010E956F95510A0A38E030
:10402C0095C100F0000E016E026E036E003600901A
:10403C00013602360336003600900136023603365E
:10404C006C0E0024F66E560E0120F76E000E022048
:10405C00F86E09006F00D4FF01F009006F00D4FF67
:10406C0002F009006F00D4FF03F009006F00D4FFC9
:10407C0004F00450A35D08E10350A25D05E1025079
:10408C00A15D02E10150A05D01E202D0952BC5D7E4
:10409C008BD0010E956F9551080A38E095C100F050
:1040AC00000E016E026E036E003600900136023671
:1040BC00033600360090013602360336020E002419
:1040CC00F66E570E0120F76E000E0220F86E0900F6
:1040DC006F00D4FF01F009006F00D4FF02F009005B
:1040EC006F00D4FF03F009006F00D4FF04F00450FC
:1040FC00A35D08E10350A25D05E10250A15D02E160
:10410C000150A05D01E202D0952BC5D74DD0010E18
:10411C00956F95510C0A38E095C100F0000E016EB8
:10412C00026E036E003600900136023603360036FE
:10413C000090013602360336D40E0024F66E4B0E78
:10414C000120F76E000E0220F86E09006F00D4FFFC
:10415C0001F009006F00D4FF02F009006F00D4FFDA
:10416C0003F009006F00D4FF04F00450A35D08E1D4
:10417C000350A25D05E10250A15D02E10150A05D7A
:10418C0001E202D0952BC5D70FD00550000AD8B448
:10419C0042D70550C00AD8B43ED70550800AD8B4CF
:1041AC0078D70550400AB3E0800E006E800E94194B
:1041BC00005C02E19351955D03E293C195F10DD042
:1041CC00800E9419006E800E005C02E19551935D97
:1041DC0004E295C193F1000E946F965197110EE085
:1041EC00030E9815006E99C101F0000E01160050D7
:1041FC00011004E0010E965F000E975B800E94197F
:10420C00006E800E9719005C02E19651935D05E2F9
:10421C009351965F9451975B02D0966B976BC40E3B
:10422C009815016E9951080B026E0250080A02E1B2
:10423C00400E011808E19651971104E0010E965FAB
:10424C00000E975B1CD0C00E9815016E9951080B8F
:10425C00026E0250080A02E1800E011810E1800E75
:10426C00006E800E9719005C02E19651020805E27F
:10427C00020E965F000E975B02D0966B976B98A51B
:10428C0069D098A315D098A103D02D0E8F6F02D0B2
:10429C002B0E8F6F600013F6E1FF600017F6E2FF44
:1042AC0060003FF6E6FF844B852BA44BA52B3BD03F
:1042BC0098A10DD0600013F6E1FF600017F6E2FF45
:1042CC00200EE66E844B852BA44BA52B2CD0C00E58
:1042DC009815016E9951080B026E0250080A02E102
:1042EC00800E011820E1600013F6E1FF600017F664
:1042FC00E2FF300EE66E844B852BA44BA52B98ABBE
:10430C0003D0580E906F02D0780E906F600013F6A9
:10431C00E1FF600017F6E2FF600043F6E6FF844B16
:10432C00852BA44BA52B9651971113E0600013F627
:10433C00E1FF600017F6E2FF300EE66E844B852B32
:10434C00A44BA52B010E965F000E975B965197110F
:10435C00EDE182D09651971115E098B713D060001B
:10436C0013F6E1FF600017F6E2FF200EE66E844BB9
:10437C00852BA44BA52B010E965F000E975B9651D7
:10438C009711EDE198A315D098A103D02D0E916F44
:10439C0002D02B0E916F600013F6E1FF600017F650
:1043AC00E2FF600047F6E6FF844B852BA44BA52B60
:1043BC000ED098A10CD0600013F6E1FF600017F648
:1043CC00E2FF200EE66E844B852BA44BA52BC00E72
:1043DC009815016E9951080B026E0250080A02E101
:1043EC00400E01180DE1600013F6E1FF600017F6B6
:1043FC00E2FF300EE66E844B852BA44BA52B2CD004
:10440C00C00E9815016E9951080B026E0250080AE5
:10441C0002E1800E011820E1600013F6E1FF60005C
:10442C0017F6E2FF300EE66E844B852BA44BA52BC2
:10443C0098AB03D0580E926F02D0780E926F60003A
:10444C0013F6E1FF600017F6E2FF60004BF6E6FFA3
:10445C00844B852BA44BA52B800E006E800E9419DB
:10446C00005C02E19351955D0DE2600013F6E1FFF3
:10447C00600017F6E2FF300EE66E844B852BA44BE2
:10448C00A52BEAD793C100F094C101F0010E935F04
:10449C00000E945B00500110D8B43FD1C00E98159B
:1044AC00006E00C0A6F11CD193C100F094C101F0C4
:1044BC00000E94BFFF0E026E036E003600900136A4
:1044CC0002360336003600900136023603366C0E87
:1044DC000024F66E560E0120F76E000E0220F86EC8
:1044EC0009006F00D4FF04F009006F00D4FF05F041
:1044FC0009006F00D4FF06F009006F00D4FF07F02D
:10450C00A0C100F0A1C101F0A2C102F0A3C103F04F
:10451C00CDEC0FF00A0E046E000E056E066E076EE3
:10452C00CDEC0FF008C000F009C001F00AC002F099
:10453C000BC003F0300E0024956FE1D098AB4AD03D
:10454C0093C100F094C101F0000E94BFFF0E026EF7
:10455C00036E0036009001360236033600360090AA
:10456C00013602360336020E0024F66E570E012079
:10457C00F76E000E0220F86E09006F00D4FF04F0F5
:10458C0009006F00D4FF05F009006F00D4FF06F09E
:10459C0009006F00D4FF07F0A0C100F0A1C101F029
:1045AC00A2C102F0A3C103F0CDEC0FF00F0E001668
:1045BC00000E0116021603165D0E0024F66E580E40
:1045CC000120F76E000E0220F86E09006F00D4FF78
:1045DC0095F149D093C100F094C101F0000E94BF45
:1045EC00FF0E026E036E0036009001360236033663
:1045FC0000360090013602360336020E0024F66EA9
:10460C00570E0120F76E000E0220F86E09006F00A5
:10461C00D4FF04F009006F00D4FF05F009006F000F
:10462C00D4FF06F009006F00D4FF07F0A0C100F022
:10463C00A1C101F0A2C102F0A3C103F0CDEC0FF0B7
:10464C000F0E0016000E0116021603164C0E002457
:10465C00F66E580E0120F76E000E0220F86E09005F
:10466C006F00D4FF95F14BD093C100F094C101F0D1
:10467C00000E94BFFF0E026E036E003600900136E2
:10468C000236033600360090013602360336D40E5D
:10469C000024F66E4B0E0120F76E000E0220F86E11
:1046AC0009006F00D4FF04F009006F00D4FF05F07F
:1046BC0009006F00D4FF06F009006F00D4FF07F06B
:1046CC00A0C100F0A1C101F0A2C102F0A3C103F08E
:1046DC00CDEC0FF0070E0014956F300E95270FD010
:1046EC00A651000AD8B4E0D6A651C00AD8B4DCD67C
:1046FC00A651800AD8B422D7A651400AB5E0600072
:10470C0013F6E1FF600017F6E2FF600057F6E6FFD4
:10471C00844B852BA44BA52BB5D698A71CD0800E0B
:10472C00006E800E9719005C02E19651000813E2AE
:10473C00600013F6E1FF600017F6E2FF200EE66E54
:10474C00844B852BA44BA52B010E965F000E975B1B
:10475C0096519711EDE13BEF12F0A4C100F0A5C109
:04476C0001F0120046
:10477000200E0101626F230E636F840E646F010EC1
:10478000656F3E01F86BF96BFA6BFB6BEC0EFD1776
:08479000F889F885F88F12008A
:10479800760E0101826F010E836F71C184F172C1BF
:1047A80085F173C186F174C187F175C188F1820EF4
:1047B800896F010E8A6F36EC12F000C080F101C0DB
:1047C80081F100507125E16E01507221E26EE66AB6
:0A47D80080C100F081C101F0120061
:1047E200A08CA09CA08CA16A080EA36EFF0E9F6EE7
:0E47F2009E6A3901A791600EA06EA08E120083
:1048000071C1B1F172C1B2F173C1B3F10101B46B05
:06481000AEEC02F0120004
:10481600800E6E6ECC0E6D6E800E6C6E6E983F01C5
:084826005F835F916E8E1200AA
:10482E000050086E0150006E016A026A036A0B6A3C
:10483E000C6A960E036E0A6A00C001F008C000F002
:0A484E00086A026AE8EC11F012009B
:10485800596A5A6A000E5A5C02E17F0E595C18E2E6
:104868005B0E5924E16E000E5A20E26E6F0087FF3E
:10487800E1FF6F008BFFE2FFE66A010E5924006E2C
:10488800000E5A20016E00C059F001C05AF0E2D75C
:104898005B6A596A5A6A576A586A536A546A556A07
:1048A800566A01014D6B3D01F289F96BFA6B3901CA
:0448B80093871200D0
:0648BC00A3EC11F0120054
:1048C20071C102F072C103F002C000F003C001F036
:1048D200024A032A600003F0E9FF600007F0EAFFE2
:1048E200EE5201E0F1D701017151025C006E72518A
:0E48F2000358016E010E005E000E015A120006
:0E49000037DF71C184F190EC11F0F89F1200C6
:10490E0009006F00D7FFE6FF0006FAE10106F8E1A5
:02491E00120085
:104920006000C7F5F6FF6000CBF5F7FF6000CFF53C
:10493000F8FF09006F00D4FF00F0005216E060009D
:10494000C7F5F6FF6000CBF5F7FF6000CFF5F8FF85
:1049500009006F00D4FFB5F191EC01F0010E0101E7
:0C4960007127000E72237323DBD71200B6
:10496C00FF0ECA6E3A014083830EC26EC296C29885
:10497C00C294BA86BA88BA84C296BA96506BCB6A7D
:10498C00FF0EC36EFF0E516F3E01BC6BB86BCC6A51
:10499C003A01606B800EC46EC296BA963E01C16B32
:0849AC00C19FC183C1911200FB
:1049B40024EC12F0BC0E0101846F480E856F000ECA
:1049C400866F000E876F220E886F030E896FB50EF7
:1049D4008A6F010E8B6FFF0E8C6FFF0E8D6F000EB2
:1049E4008E6F000E8F6FC40E906F000E916F000ECD
:1049F400926F000E936F6FEC11F0846B856BA9ECD2
:044A040011F012009B
:104A08000D0E0101B56F91EC01F00A0E0101B56FB1
:064A180091EC01F0120018
:104A1E00520E0B6E2B0E0C6E000E0D6E0D2EFED763
:0C4A2E000C2EFCD70B2EFAD70000120053
:104A3A006000C7F5E9FF6000CBF5EAFF6F00B8FF39
:104A4A0073F1000E0101746F000E746F000E741979
:104A5A0002E1200E731907E0000E741902E1090E33
:104A6A00731901E003D0714B722BE2D7756B766B29
:104A7A00776B786B000E741902E12D0E731905E13C
:104A8A00774B782B714B722B08D0000E741902E108
:104A9A002B0E731902E1714B722B6000C7F5E9FF07
:104AAA006000CBF5EAFF6F00B8FF73F1000E746F78
:104ABA00000E746F73C1ACF16AEC0EF0005219E08B
:104ACA0075C100F076C101F00A0E046E000E056E83
:104ADA0043EC11F0300E735D026E000E7459036ED2
:104AEA0002500024756F03500120766F714B722BB0
:104AFA00D4D77751781108E075510008006E76C155
:104B0A0001F0000E015604D075C100F076C101F023
:024B1A00120087
:0E4B1C0071C184F172C185F1C9EC11F0120073
:104B2A006000C7F5E9FF6000CBF5EAFFEE5215E039
:104B3A006000C7F5E9FF6000CBF5EAFF6000CFF53A
:104B4A00D9FF6000D3F5DAFFEE50DE1806E1010165
:104B5A00714B722B734B742BE3D76000C7F5E9FFD7
:104B6A006000CBF5EAFF6000CFF5D9FF6000D3F50E
:104B7A00DAFFDE50EE5C006E016A000E015A120086
:104B8A00FF0E01017115036E7251030B046E03C00F
:104B9A0000F004C001F001320032019E01320032FD
:104BAA00019E600003F06DFF030E7115026E060E82
:104BBA00016E02C000F0015004E000360090FF0FC1
:0A4BCA00FBD7600003F06CFF12003F
:104C040000C01AF001C019F03901A3A776D093A708
:104C140074D052DE00C04DF13D01F9AB0FD0F99BC9
:104C2400010E01015825006E000E5921016E00C0CD
:104C340058F101C059F16F00A0F74DF13D01F9A7FA
:104C44000ED0010E01015825006E000E5921016E8F
:104C540000C058F101C059F12FDE00C04DF101012F
:104C64004D510D0A07E05850000802E157507F08E3
:104C740001E324D0010E556E000E566E5B0E5924CE
:104C8400E16E000E5A20E26E6F0087FFE1FF6F00B5
:104C94008BFFE2FFE66A3901939759C057F05AC077
:104CA40058F0596A5A6A5850000802E157507F0870
:104CB40004E2020E556E000E566E1FD0556A566AF7
:104CC4005B0E5924E16E000E5A20E26E6F0087FFDE
:104CD400E1FF6F008BFFE2FF600037F5E6FF59C08C
:104CE40057F05AC058F0010E5924006E000E5A2095
:104CF400016E00C059F001C05AF01AC000F019C08A
:044D040001F01100A9
:104D080041EC2CF0600E3901D96F080EDF6F6E0090
:104D180070F74EF1000E01014F6F24DE01014B6B5D
:104D28004C6B800E4C19006E800E005C02E1200E68
:104D38004B5D10E2DB0E4B25E16E000E4C21E26E5E
:104D48006F0087FFE1FF6F008BFFE2FFE66A4B4BC6
:104D58004C2BE7D74B6B4C6B800E4C19006E800EBA
:104D6800005C02E1500E4B5D10E2FB0E4B25E16E3C
:104D7800000E4C21E26E6F0087FFE1FF6F008BFF92
:104D8800E2FFE66A4B4B4C2BE7D7596A5A6A576AD7
:104D9800586AFB0E4B6E000E4C6E3D01F38F400EB1
:104DA800F56F030EF66FF28F01DEBC0E0101846F02
:104DB800480E856F000E866F000E876F220E886F73
:104DC800030E896FB50E8A6F010E8B6FFF0E8C6F05
:104DD800FF0E8D6F000E8E6F000E8F6FC40E906FDA
:104DE800000E916F000E926F000E936F6FEC11F032
:104DF800110E0B6E3C0E0C6ECB0E0D6E0D2EFED7EB
:104E08000C2EFCD70B2EFAD70C0EB56F91EC01F0D7
:104E1800F7DD050E0101716F580E726F000E736F8A
:104E28007BDD760E0101716F570E726F000E736F86
:104E380073DDFA0E0101716F540E726F000E736FFD
:104E48006BDD350E0101716F550E726F000E736FB9
:104E580063DD6F0E0101716F550E726F000E736F77
:104E68005BDD100E0101716F560E726F000E736FCD
:104E780053DD3B0E0101716F580E726F000E736F98
:104E88004BDD000E4D6EFA0E4E6E4BC071F14CC0EC
:104E980072F1E10E0101736F560E746F000E756F9B
:104EA800000E766FFA0E776F73DC4BC071F14CC051
:104EB80072F130DE1B0E716F000E726F2BDEABDDF0
:104EC8007D0E716F580E726F000E736F25DDA3DDB6
:104ED8000A0E476E000E486EBA86800E006E800E6F
:104EE8004818005C02E14750000813E2BC7A150E2E
:104EF8000B6E4B0E0C6EBE0E0D6E0D2EFED70C2ECD
:104F0800FCD70B2EFAD70000010E475E000E485A58
:104F1800E4D7BA9680DD28DC010E0101716FECDC64
:104F280000C049F001C04AF05294376A386A01015A
:104F38004B6B4C6B516A400E716F560E726F000EC0
:104F4800736FEADCA0EC01F00E0E0101716F726B59
:104F5800150E736F51DC95EC01F05E0E0101716F57
:104F6800570E726F000E736FD7DC37DCC80E356EC4
:104F7800000E366EBC0E0101716F560E726F000E78
:104F8800736FCADC44DC47DDF30E0101716F570E05
:104F9800726F000E736FC0DCBA86800E0101716FEC
:104FA800000E726FEEDD37DDBA96290E716F580E5E
:104FB800726F000E736FB0DCF40E0101716F010E99
:104FC800726FDFDD28DDBA96BA86170E716F580E3C
:104FD800726F000E736FA0DC200E0101716F030E5B
:104FE800726FCFDD18DDBA96BA86CC0E716F570E88
:104FF800726F000E736F90DCE80E0101716F030E83
:10500800726FBFDDBA96FCDC06DDC80E356E000E89
:10501800366E8C0E0101716F570E726F000E736F32
:105028007BDC4F6A506A39019387939FD28E596A05
:105038005A6A576A586A556A566A940E0101716F1E
:10504800560E726F000E736F67DCBA8601DCBA9673
:10505800010E0101716F50DC00C049F001C04AF037
:105068003950010A13E149C000F04AC001F0013289
:105078000032019E01320032019E00C035F001C0AD
:1050880036F000C071F101C072F17BDD0101FB0E49
:105098004B6E000E4C6E35C000F036C001F017ECB8
:1050A80024F0DE0E046EFF0E056E470E066E7B0EB4
:1050B800076EAFEC01F000C069F101C06AF102C0EF
:1050C8006BF103C06CF14BC071F14CC072F1480E2A
:1050D800736F540E746F000E756F4BC176F14CC12F
:1050E80077F149C078F14AC079F149C07AF14AC0EC
:1050F8007BF100C07CF101C07DF102C07EF103C0EC
:105108007FF1CCEC23F04BC071F14CC072F102DDA1
:10511800800E006E800E5018005C02E14F500008AF
:1051280015E24BC071F14CC072F16E0E736F580EE0
:10513800746F000E756F4FC076F150C077F1CCECEC
:1051480023F04BC071F14CC072F1E4DC59DC520E13
:105158000B6E2B0E0C6E000E0D6E0D2EFED70C2E48
:10516800FCD70B2EFAD70000000E561802E1010EEC
:105178005518D8A43DD1FB0E4B6E000E4C6E4BC09B
:1051880071F14CC072F1B70E0101736F570E746F55
:10519800000E756F5B0E766F000E776FCCEC23F008
:1051A8004BC071F14CC072F1B5DC5B50430AD8A416
:1051B8009BD0000E006E5850005C02E15750010869
:1051C800D8B092D001015C0E716F000E726F61EC65
:1051D80024F000C067F101C068F1010E4B6F000EAA
:1051E8004C6F800E4C19006E800E6819005C02E14D
:1051F80067514B5D1CE25B0E4B25E96E000E4C219E
:10520800EA6E6F00A7FFE9FF6F00ABFFEAFF6F00D0
:10521800B8FF00F000C066F166C1ACF16AEC0EF0B0
:105228000050000A01E103D04B4B4C2BDAD74C510C
:10523800681902E167514B1956E15C0E716F000E57
:10524800726F1DEC25F000C067F101C068F1800E97
:10525800026E800E0118025C02E1005000080FE2A5
:10526800800E6819006E800E040A005C02E1000ED0
:10527800675D05E267C135F068C136F002D0356A6E
:10528800366ABA86396AA20E716F570E726F000EAF
:10529800736F90EC24F035C071F136C072F171DC97
:1052A800BA964BC071F14CC072F1220E736F570E53
:1052B800746F000E756F35C076F136C077F1CCEC9F
:1052C80023F04BC071F14CC072F124DCA30E0B6EBD
:1052D800570E0C6E020E0D6E0D2EFED70C2EFCD73F
:1052E8000B2EFAD70000666B5B50410A13E1000EE3
:1052F800006E5850005C02E1575000080BE20101B3
:10530800E00E716F570E726F000E736F90EC24F001
:10531800010E396E5B0E0101716F000E726F410E46
:10532800736F000E746F95EC25F000C06FF101C02B
:1053380070F1000E011802E1000E001857E101019A
:10534800676B686B800E6819006E800E030A005C3C
:1053580002E1F00E675D1BE267C16DF168C16EF195
:1053680067C171F168C172F10CDC020E0B6EA00E00
:105378000C6E920E0D6E0D2EFED70C2EFCD70B2E3A
:10538800FAD70000100E6727000E6823DBD7FF0E40
:10539800676F030E686F800E006E800E6819005CE0
:1053A80002E1675110081CE267C16DF168C16EF136
:1053B80067C171F168C172F1C5EC25F0020E0B6E80
:1053C800A00E0C6E920E0D6E0D2EFED70C2EFCD775
:1053D8000B2EFAD70000100E675F000E685BDBD754
:1053E80035C071F136C072F1C5EC25F0556A566AC0
:1053F800000E561802E1020E55181DE10101FB0EC0
:105408004B6E000E4C6E4BC071F14CC072F1410EE8
:10541800736F570E746F000E756F57C076F158C0D2
:1054280077F1CCEC23F04BC071F14CC072F18EECEB
:1054380025F0556A566A01014B4B4C2B06D6FFD70F
:1054B40000C018F0390193AF1BD0A3AF19D0000E70
:1054C400006E3850005C02E13750000811E23C0ED7
:1054D400B76EB00EB66E374A382A000E006E3850DA
:1054E400005C02E13750090802E25284939FA39FB3
:0654F40018C000F01100D9
:1058820010EE1BF02C0E006E010E016E880EF66EED
:0E589200540EF76E000EF86E87EC24F0120034
:104BD4000100000008000000400000000002000086
:104BE400001000000080000000000400000020000D
:104BF4000000000100000008000000400000000068
:10544800204D65737572652023253564203D3E2007
:105458004144432031326220524131203D202025F1
:105468002035642020736F697420307825303458D3
:105478002020447574793D25332E3166202525007A
:105488002056657269666965206C6120736F727455
:0A549800696520524335200D0A001B
:0254A200000008
:0254A400000006
:0154A6000104
:0754A700286E756C6C2900F2
:0654AE0052414D50450083
:1054FA00204469726563746F7279203A20433A5C7A
:10550A005F4D696B726F435C5F4D657350726F6A72
:10551A006574735F4D696B726F435C5F31384632F5
:0B552A00374B34325F50574D0D0A0024
:105535002050726F6A6574203A2031384632374BF5
:1055450034325F55415254315F52585F49545F417F
:105555004443305F50574D5F426173655F3230326F
:0A556500312E6D637070690D0A00AD
:10556F0020536F75726365203A205F3138463237AA
:10557F004B34325F33324D687A5F55617274315FED
:10558F004144435F50574D5F3130625F32303231AB
:09559F00303531372E630D0A008E
:1055A8000000007FCDCC4C7B0AD723786F1203759F
:1055B80017B75171ACC5276EBD37066B95BF5667D7
:1055C80077CC2B645F700961FFE65B5D08E53C3CC6
:0455D8006042221BF0
:1055DC000000007F000020820000488500007A88CF
:1055EC0000401C8C0050438F0024749280961896B7
:1055FC0020BC3E99286B6E9CF90215A0EC782DC14D
:04560C00CAF249E2B3
:1056100020434F4E464947203A20503138463236D3
:105620004B32325F464F53435F696E7465726E65ED
:105630005F36344D687A2E6366677363680D0A00BF
:10564000204166666563746174696F6E20285050EE
:1056500053292050494E2052433220E020536F728C
:0C5660007469652050574D35200D0A007C
:10566C00010000000A00000064000000E8030000D4
:10567C0010270000A086010040420F008096980081
:08568C0000E1F50500CA9A3B9C
:10569400202D2D2D2D2D2D2D2D2D2D204D61696E7F
:1056A40020626F75636C652D2D2D2D2D2D2D2D2DC7
:0856B4002D2D2D2D200D0A0003
:1056BC0020496E69742050573520313062697473FB
:1056CC002061742031303030487A206F6E20524384
:0556DC0035200D0A005D
:1056E10020436C6F636B20696E697469616C65201E
:1056F100696E204B687A203D2025303575200D0AD2
:0157010000A7
:105702000100000010000000000100000010000075
:105712000000010000001000000000010000001065
:10572200204E65772049526174696F2028313020FC
:0F5732006269747329203D20253564200D0A001B
:105741004275666665723120554152543120467565
:0D5751006C6C203D2025303564200D0A00D1
:10575E0020496E69742054696D6572342020464F5D
:08576E0053432F34200D0A0003
:1057760020506F77657220737570706C793A20339C
:065786002E36560D0A004C
:10578C002020496E746572727570747320696E692D
:06579C007473200D0A00E9
:1057A2000D0A20204B6579626F617264204D6F642F
:0557B20065200D0A0056
:1057B700205265636570742055415254313D202550
:0557C70073200D0A0033
:1057CC0020205057352076616C75653D3130303076
:0457DC00200D0A0092
:1057E0000D0A2020416E616C6F67204D6F6465204B
:0357F0000D0A009F
:1057F30020205057352076616C75653D3132380D68
:025803000A0099
:10580500204D4355203A2031384632374B34320D3E
:025815000A0087
:1058170020205057352076616C75653D3830300D46
:025827000A0075
:1058290020205057352076616C75653D3530300D37
:025839000A0063
:10583B0020464F534320203A2036344D487A0D0AE8
:01584B00005C
:10584C0030313233343536373839616263646566EA
:01585C00004B
:10585D003031323334353637383941424344454699
:01586D00003A
:0F586E002020657272657572203D20253564001B
:05587D00476F0D0A0059
:020000040030CA
:0A000000042BFFBF0B3F9F0F010010
:00000001FF
